:020000040000FA
:020000000528D1
:0800080004288501870107307F
:100010009900831681013C308500143095008701DA
:100020008312A001A101A201A301A4013F30870016
:10003000A00A0130051D023020020319A001031996
:10004000A10A0A3021020319A1010319A20A0A30E8
:1000500022020319A2010319A30A0A302302051977
:1000600007100319A3010319A40A0A302402031973
:10007000A40101302002A50C02302102A50C02309F
:100080002202A50C02302302A50C02302402A50C8A
:10009000051D071001302402A50C0314A50C031440
:1000A000A50C250900007220722072207220722097
:1000B00073207520051A17288514051E5D28051460
:1000C000A001A101A201A301A4013F308700A00A61
:1000D0000130051D0230200285196C28851D6E280F
:1000E00085101D28732874287528080044004600D0
:1000F0004400490056002E00610073006D0020008E
:10010000560065007200200031002E0030003000E3
:100110002C0020005200690063006800610072003A
:1001200064002000480020004D00630043006F0081
:1001300072006B006C00650020003200300030005F
:040140003600200065
:02400E00833FEE
:00000001FF
